:020000040000FA
:060000003BEF1AF01200B4
:060008008FEF13F012005F
:06002A000200AD330000EE
:10003000FD00000001000000A234000000000000EC
:0400400018000000A4
:0C0044000001EA6BEB6B8A6A896AF90E16
:10005000926E010EC26E0E0EC16E860EC06EBD6A2D
:10006000010E066E640EEC6FD00EEF6F070EF06F90
:10007000080EED6F0B0EEE6F000E036E046A096E34
:100080000A6A076E086A800ED56E1200F2A418D0B4
:10009000F2940001EB2B050E0101405D07E20A0E10
:1000A0000001EB5D03E38974EB6B1200050E0101A7
:1000B000405D06E12E0E0001EB5D02E38974EB6BFF
:1000C0001200E4DF050E0101405D45E36D50020BB7
:1000D00001E012000001EA5129E0800E04010C1534
:1000E00025E1400EE66E600EE66E000EE66EA0ECB8
:1000F00014F0E552E552E5520001EA6B016A025044
:10010000015C13E20150EA6AE00FE96E000EEA2298
:10011000EF50E66E0150EA6A600FE96E000EEA22C7
:10012000E552E750EF6E012AEAD7026A0001FD515D
:10013000005C10E3400EE66EA00EE66E000EE66E6A
:10014000E2EC14F0E552E552E5520001FD6FE85093
:1001500001E0006A01D81200D9CFE6FFE1CFD9FF54
:10016000090EE1260001FD51005C02E34FEF13F0A0
:100170000001EA5102E04FEF13F089820050EA6A71
:10018000A00FE96E000EEA22EF50F10A02E102EF41
:1001900013F0010A02E1C5EF12F0020A02E1A8EF32
:1001A00012F0CF0A02E15DEF12F0010A02E119EF4D
:1001B00012F0070A02E110EF12F0010A02E1C7EFA4
:1001C00011F0030A02E179EF11F0010A02E168EF90
:1001D00011F00F0A02E13FEF11F0010A02E1F2EF24
:1001E00010F0030A02E1CAEF10F0010A02E15BEF2E
:1001F00010F0070A02E1DCEF0FF0010A02E1A3EFC1
:100200000FF0030A02E16CEF0FF0010A02E131EF97
:100210000FF01F0A02E1DCEF0EF0020A02E167EFC5
:100220000EF0030A02E1CCEF0DF0020A02E125EF25
:100230000DF0070A02E1EDEF0CF0010A02E19AEF7E
:100240000CF0030A02E149EF0CF0010A02E1C8EFE9
:100250000BF00F0A02E148EF0BF0010A02E1EDEFAB
:100260000AF0030A02E1A6EF0AF0010A02E140EFF8
:100270000AF0070A02E10AEF0AF0010A02E1D4EFEC
:1002800009F0030A02E18EEF09F0010A02E10DEF25
:1002900008F03F0A02E1DCEF07F0010A02E1C2EFD9
:1002A00007F0030A02E1A6EF07F0010A02E18CEF72
:1002B00007F0070A02E170EF07F0010A02E152EFCE
:1002C00007F0030A02E136EF07F0010A02E11CEF32
:1002D00007F00F0A02E1D3EF06F0010A02E1BAEFDC
:1002E00006F0030A02E170EF06F0010A02E128EFCE
:1002F00006F0070A02E1CBEF05F0010A01E1EDD3B8
:10030000030A01E190D3010A01E174D31F0A01E15C
:10031000F5D2010A01E1A6D2030A01E119D2010ACC
:1003200001E1F5D1070A01E1C3D1010A01E1A8D138
:10033000030A01E18FD1010A01E176D10F0A01E13F
:10034000F5D0010A01E1E6D0030A01E1C1D0010ABA
:1003500001E19BD0070A67E0010A43E0030A0AE0D3
:10036000010A02E048EF13F0E66A5AEC13F0E55296
:100370004DEF13F0010EE66E5AEC13F0E55262DE1B
:10038000E66A5AEC13F0E552060EE66E5AEC13F0EC
:10039000E552010EE66E5AEC13F0E552E66A5AECAD
:1003A00013F0E552E66A5AEC13F0E552020EE66EDF
:1003B0005AEC13F0E552200EE66E5AEC13F0E552BB
:1003C000520EE66E5AEC13F0E552530EE66E5AECFE
:1003D00013F0E552540EE66E5AEC13F0E5524DEF71
:1003E00013F0020EE66E5AEC13F0E552E66A5AEC90
:1003F00013F0E552060EE66E5AEC13F0E552010ECC
:10040000E66E5AEC13F0E552E66A5AEC13F0E55248
:10041000E66A5AEC13F0E552020EE66E5AEC13F05F
:10042000E5524DEF13F0030EE66E5AEC13F0E55271
:100430000028186E0001FD51185C18E2002A0050D7
:10044000EA6AA00FE96E000EEA22EFCFDFFF3D0E51
:10045000DF5C06E2DFCFE6FF5AEC13F0E55205D091
:10046000FE0EE66E5AEC13F0E5520DD0FE0EE66E6F
:100470005AEC13F0E5520028EA6AA00FE96E000E6C
:10048000EA22040EEF6E4DEF13F0400E015C09E21C
:100490000150EA6A600FE96E000EEA22EF6A012A53
:1004A000F4D7016A04010CBF0CD0400EE66E600E5A
:1004B000E66E000EE66EA0EC14F0E552E552E55251
:1004C00003D00001010EEA6FFDC000F04DEF13F004
:1004D000050EE66E5AEC13F0E552000E036E046A48
:1004E000096E0A6A076E086A840ECB6E040ECA6E25
:1004F0009E909D80F40ECF6E480ECE6E810ECD6E16
:10050000BE6A0C0EBD6E9494C00EF26E1E0ED26EBC
:100510004DEF13F0060EE66E5AEC13F0E5529D9087
:10052000CD6ABD6A0E0ED26E4DEF13F0070EE66E69
:100530005AEC13F0E552030E0024186E0001FD5131
:10054000185C63E2002A0050EA6AA00FE96E000E10
:10055000EA22EF500D6E0D50030A40E0010A2BE035
:10056000030A16E0010A01E04CD0002A0050EA6AB2
:10057000A00FE96E000EEA22EF50066E002A00502E
:10058000EA6AA00FE96E000EEA22EFCFECF03CD051
:10059000002A0050EA6AA00FE96E000EEA22EFCFAF
:1005A000F0F0002A0050EA6AA00FE96E000EEA227D
:1005B000EFCFEFF029D0002A0050EA6AA00FE96ED1
:1005C000000EEA22EFCFF2F0002A0050EA6AA00FF4
:1005D000E96E000EEA22EFCFF1F016D0002A0050AB
:1005E000EA6AA00FE96E000EEA22EFCFEDF0002AD2
:1005F0000050EA6AA00FE96E000EEA22EFCFEEF09B
:1006000003D0020E002600D00DD0FE0EE66E5AEC8E
:1006100013F0E5520028EA6AA00FE96E000EEA2204
:10062000040EEF6E4DEF13F0080EE66E5AEC13F069
:10063000E552F29E06500D6E0D5009E000000000DC
:10064000000000000000000000000D06F5D7F28E4B
:100650004DEF13F0090EE66E5AEC13F0E552F29EE0
:10066000ECC00DF00D5009E000000000000000009B
:100670000000000000000D06F5D7F28E4DEF13F0DC
:100680000A0EE66E5AEC13F0E552F29EEFC013F03C
:10069000F0C014F01350141008E000000000000037
:1006A00000001306000E145AF5D7F28E4DEF13F02A
:1006B0000B0EE66E5AEC13F0E5520028186E00019E
:1006C000FD51185C15E2002A0050EA6AA00FE96E9D
:1006D000000EEA22EF500D6E0D5009E00000000000
:1006E000000000000000000000000D06F5D70DD04E
:1006F000FE0EE66E5AEC13F0E5520028EA6AA00FEF
:10070000E96E000EEA22040EEF6E4DEF13F0A19495
:100710000C0EE66E5AEC13F0E552C282C2B2FED75E
:10072000A1A40AD0E66A5AEC13F0E552E66A5AEC44
:1007300013F0E5524DEF13F0C450E66E5AEC13F08F
:10074000E552C350E66E5AEC13F0E5524DEF13F04C
:100750000D0EE66E5AEC13F0E5520028186E0001FB
:10076000FD51185C70E29D50400B03E0D250200B0D
:1007700006E1FE0EE66E5AEC13F0E55263D0A1944A
:10078000002A0050EA6AA00FE96E000EEA22EF503C
:10079000136E146A13C00BF014C00CF0070E0C0299
:1007A000F3CF0CF0070E0B02F3CF0BF0F4500C2636
:1007B0000F0E0D6EE80E136E030E146E1350141010
:1007C00008E000000000000000001306000E145AAC
:1007D000F5D70D06083404E207500E08000E085441
:1007E00008E3D880085004E7F20E075CFF0E0858B3
:1007F00002E20D50DFE1A1A405D0E66A5AEC13F045
:10080000E55220D0083404E207500E08000E0854C8
:1008100008E3D880085004E7F20E075CFF0E085882
:1008200006E2FE0EE66E5AEC13F0E5520BD00050D5
:10083000EA6AA00FE96E000EEA22EF50E66E5AEC6B
:1008400013F0E5520DD0FE0EE66E5AEC13F0E552B1
:100850000028EA6AA00FE96E000EEA22040EEF6E8D
:100860004DEF13F00E0EE66E5AEC13F0E552002831
:10087000186E0001FD51185C32E2002A0050EA6A4D
:10088000A00FE96E000EEA22EF500D6E010E0D145E
:1008900002E0000E01D0010EE8B08B82E8A08B923E
:1008A000020E0D1402E0010E01D0000EE8B0948299
:1008B000E8A09492040E0D1402E0010E01D0000E87
:1008C000E8B08B80E8A08B90080E0D1402E0010EBA
:1008D00001D0000EE8B09480E8A094900DD0FE0EF8
:1008E000E66E5AEC13F0E5520028EA6AA00FE96EB2
:1008F000000EEA22040EEF6E4DEF13F00F0EE66EBF
:100900005AEC13F0E5520028186E0001FD51185CF6
:1009100062E2002A0050EA6AA00FE96E000EEA22A5
:10092000EF50010B02E0010E01D0000EE8B08A8A00
:10093000E8A08A9A0050EA6AA00FE96E000EEA2247
:10094000EF50020B02E0010E01D0000EE8B0938AD6
:10095000E8A0939A0050EA6AA00FE96E000EEA221E
:10096000EF50040B02E0010E01D0000EE8B08A8CBB
:10097000E8A08A9C0050EA6AA00FE96E000EEA2205
:10098000EF50080B02E0010E01D0000EE8B0938C8E
:10099000E8A0939C0050EA6AA00FE96E000EEA22DC
:1009A000EF50100B02E0010E01D0000EE8B08A8E6D
:1009B000E8A08A9E0050EA6AA00FE96E000EEA22C3
:1009C000EF50200B02E0010E01D0000EE8B0938E34
:1009D000E8A0939E0DD0FE0EE66E5AEC13F0E552A1
:1009E0000028EA6AA00FE96E000EEA22040EEF6EFC
:1009F0004DEF13F0100EE66E5AEC13F0E5520D6A4F
:100A00008ABA0D8093BA0D828ABC0D8493BC0D8680
:100A10008ABE0D8893BE0D8A0D50E66E5AEC13F017
:100A2000E5524DEF13F0110EE66E5AEC13F0E5525D
:100A3000020E0024186E0001FD51185C3FE2002AEE
:100A40000050EA6AA00FE96E000EEA22EFCF14F020
:100A5000002A0050EA6AA00FE96E000EEA22EFCFEA
:100A600013F0F29E8A9A8A8C8A9C8A8C8A9C8A8C41
:100A70008A9C8A8C8A9C8A8C8A9C8A8C8A9C065046
:100A80000D6E0D5009E000000000000000000000A5
:100A9000000000000D06F5D78A8C8A9C0E0E0D6EA4
:100AA00014321332819AD8B0818A818C819C0D2EA8
:100AB000F7D78A9A8A8C8A9CF28E0DD0FE0EE66E4B
:100AC0005AEC13F0E5520028EA6AA00FE96E000E16
:100AD000EA22040EEF6E4DEF13F0120EE66E5AECA2
:100AE00013F0E552020E0024186E0001FD51185C4F
:100AF00043E2002A0050EA6AA00FE96E000EEA22E3
:100B0000EFCF14F0002A0050EA6AA00FE96E000E41
:100B1000EA22EFCF13F0F29E8A9A8A8C8A9C000018
:100B20008A8A8A8C8A9C00008A9A8A8C8A9C8A8CFF
:100B30008A9C8A8C8A9C8A8C8A9C06500D6E0D50E9
:100B400009E00000000000000000000000000000BC
:100B50000D06F5D78A8C8A9C0E0E0D6E1432133258
:100B6000819AD8B0818A818C819C0D2EF7D78A9A80
:100B70008A8C8A9CF28E0DD0FE0EE66E5AEC13F033
:100B8000E5520028EA6AA00FE96E000EEA22040E80
:100B9000EF6E4DEF13F0130EE66E5AEC13F0E552C4
:100BA0000028186E0001FD51185C43E2002A005035
:100BB000EA6AA00FE96E000EEA22EFCF13F0F29E70
:100BC0008A8A8A8C8A9C8A8C8A9C00008A9A8A8C5F
:100BD0008A9C8A8C8A9C8A8C8A9C8A8C8A9C0650E5
:100BE0000D6E0D5009E00000000000000000000044
:100BF000000000000D06F5D78A8C8A9C080E0D6E49
:100C00001332819AD8B0818A818C819C0D2EF8D7BD
:100C10008A9A8A8C8A9C8A8C8A9C8A8C8A9C8A8CE6
:100C20008A9C8A8C8A9C8A8C8A9C8A8C8A9CF28E6A
:100C30000DD0FE0EE66E5AEC13F0E5520028EA6A7B
:100C4000A00FE96E000EEA22040EEF6E4DEF13F0D6
:100C5000140EE66E5AEC13F0E552F29E8A9A8A8CD4
:100C60008A9C8A8C8A9C00008A8A8A8C8A9C0000D2
:100C70008A9A8A8C8A9C8A8C8A9C8A8C8A9C938A7F
:100C800006500D6E0D5009E000000000000000004D
:100C90000000000000000D06F5D78A8C8A9C0E0E1D
:100CA0000D6E8A8C8A9CD89081BAD8801432133207
:100CB0000D2EF7D7D89014321332D8901432133245
:100CC0008A8C939A8A9CF28E14C0E6FF5AEC13F039
:100CD000E55213C0E6FF5AEC13F0E5524DEF13F066
:100CE000150EE66E5AEC13F0E552F29E8A8A8A8C53
:100CF0008A9C00008A9A8A8C8A9C00008A8A8A8C44
:100D00008A9C00008A9A8A8C8A9C8A8C8A9C8A8C0B
:100D10008A9C938A06500D6E0D5009E00000000079
:100D2000000000000000000000000D06F5D78A8CCE
:100D30008A9C080E0D6E8A8C8A9CD89081BAD880C5
:100D400013320D2EF8D78A8C8A9C8A8C8A9C8A8CC6
:100D50008A9C8A8C8A9C8A8C8A9C8A8C8A9C8A8CA3
:100D6000939A8A9CF28E13C0E6FF5AEC13F0E55278
:100D70004DEF13F0160EE66E5AEC13F0E552F29EAC
:100D80008A9A8A8C8A9C00008A8A8A8C8A9C8A8C9D
:100D90008A9C8A9A8A8C8A9C8A8C8A9C8A8C8A9C55
:100DA000F28E4DEF13F0170EE66E5AEC13F0E5528B
:100DB0000028186E0001FD51185C2FE2F29E002AF7
:100DC0000050EA6AA00FE96E000EEA22EFCF13F09E
:100DD0000001135020E08A9A8A8C8A9C00008A8A3B
:100DE0008A8C8A9C8A8C8A9C8A9A8A8C8A9C8A8C15
:100DF0008A9C8A8C8A9C06500D6E0D5009E000007A
:100E00000000000000000000000000000D06F5D703
:100E100000011306DDD7F28E0DD0FE0EE66E5AEC01
:100E200013F0E5520028EA6AA00FE96E000EEA22EC
:100E3000040EEF6E4DEF13F0180EE66E5AEC13F041
:100E4000E552F29E8A9A8A8C8A9C8A8C8A9C8A8C29
:100E50008A9C00008A8A8A8C8A9C00008A9A8A8CE2
:100E60008A9C8A8C8A9CF28E4DEF13F0190EE66EE6
:100E70005AEC13F0E552F29E8A8A8A8C8A9C000012
:100E80008A9A8A8C8A9C8A8C8A9C00008A8A8A8C9C
:100E90008A9C00008A9A8A8C8A9C8A8C8A9CF28E10
:100EA0004DEF13F01A0EE66E5AEC13F0E552F29E77
:100EB0008A9A8A8C8A9C00008A8A8A8C8A9C000082
:100EC0008A9A8A8C8A9C00008A8A8A8C8A9C000072
:100ED0008A9A8A8C8A9C8A8C8A9CF28E4DEF13F0B7
:100EE0001B0EE66E5AEC13F0E552F29E8A8A8A8C4B
:100EF0008A9C8A8C8A9C00008A9A8A8C8A9C000030
:100F00008A8A8A8C8A9C00008A9A8A8C8A9C8A8C1B
:100F10008A9CF28E4DEF13F01C0EE66E5AEC13F025
:100F2000E552F29E8A9A8A8C8A9C00008A8A8A8C70
:100F30008A9C8A8C8A9C8A8C8A9C00008A9A8A8CD9
:100F40008A9C8A8C8A9CF28E4DEF13F01D0EE66E01
:100F50005AEC13F0E552F29E8A8A8A8C8A9C000031
:100F60008A9A8A8C8A9C8A8C8A9C8A8C8A9C0000A9
:100F70008A8A8A8C8A9C00008A9A8A8C8A9CF28E41
:100F80004DEF13F01E0EE66E5AEC13F0E552F29E92
:100F90008A9A8A8C8A9C8A8C8A9C8A8C8A9C000079
:100FA0008A8A8A8C8A9C8A8C8A9C00008A9A8A8C7B
:100FB0008A9CF28E4DEF13F01F0EE66E5AEC13F082
:100FC000E5520028186E0001FD51185C17E2002A56
:100FD0000050EA6AA00FE96E000EEA22EFCF13F08C
:100FE000F29E060E0D6E1332819AD8B0818A818CE2
:100FF000819C0D2EF8D78A9AF28E0DD0FE0EE66EE9
:101000005AEC13F0E5520028EA6AA00FE96E000ED0
:10101000EA22040EEF6E4DEF13F0200EE66E5AEC4E
:1010200013F0E552020E0024186E0001FD51185C09
:1010300001E365D1002A0050EA6AA00FE96E000EB4
:10104000EA22EFCF14F0002A0050EA6AA00FE96EFE
:10105000000EEA22EFCF13F0010E13C0DBFF020EE9
:1010600014C0DBFFF29E8A9A8A8C8A9C00008A8ACE
:101070008A8C8A9C00008A9A8A8C8A9C8A8C8A9C98
:101080008A8C8A9C8A8C8A9C06500D6E0D5009E0D1
:1010900000000000000000000000000000000D063D
:1010A000F5D78A8C8A9C0E0E0D6E14321332819AFB
:1010B000D8B0818A818C819C0D2EF7D78A9A8A8C30
:1010C0008A9C030EDB6A040EDB6A030EDBCF18F08A
:1010D000040EDBCF19F00001ED51000119AE02D072
:1010E000D89003D0185C000E195801E397D08A9A63
:1010F0008A8C8A9C8A8C8A9C8A8C8A9C00008A8A28
:101100008A8C8A9C00008A9A8A8C8A9C8A8C8A9C07
:10111000ECC00DF00D5009E00000000000000000E0
:101120000000000000000D06F5D78A9A8A8C8A9C80
:1011300000008A8A8A8C8A9C8A8C8A9C8A8C8A9CE7
:1011400000008A9A8A8C8A9C8A8C8A9C06500D6E32
:101150000D5009E000000000000000000000000049
:1011600000000D06F5D78A9A8A8C8A9C8A8C8A9C04
:1011700000008A8A8A8C8A9C00008A9A8A8C8A9CBF
:101180008A8C8A9C8A8C8A9C938A06500D6E0D509C
:1011900009E0000000000000000000000000000066
:1011A0000D06F5D78A8C8A9C0E0E0D6E8A8C8A9C51
:1011B000D89081BAD880143213320D2EF7D7D89038
:1011C00014321332D890143213328A8C939A8A9C38
:1011D00006500D6E0D5009E00000000000000000F8
:1011E0000000000000000D06F5D7010EDBCF18F05F
:1011F000020EDBCF19F01350181802E11450191821
:1012000007E1030EDB500D6E030EDB68040EDB6A94
:10121000030EDB2A040E01E3DB2A57D7F28EF29E7F
:10122000D950030FE96EDACFEAFFFF0EEE1801E1A5
:10123000ED505EE10D50E66E5AEC13F0E552000100
:10124000EE510D02F350E66ED950030FE96EDACF7E
:10125000EAFFE552E750EE6EED6AD950030FE96EF2
:10126000DACFEAFFEE50ED1042E08A9A8A8C8A9C2F
:101270008A8C8A9C8A8C8A9C00008A8A8A8C8A9CA6
:1012800000008A9A8A8C8A9C8A8C8A9CECC00DF019
:101290000D5009E000000000000000000000000008
:1012A00000000D06F5D78A9A8A8C8A9C00008A8AEB
:1012B0008A8C8A9C8A8C8A9C8A8C8A9C00008A9A56
:1012C0008A8C8A9C8A8C8A9C06500D6E0D5009E08F
:1012D00000000000000000000000000000000D06FB
:1012E000F5D7030EDB06040E01E2DB06B6D705D008
:1012F000FE0EE66E5AEC13F0E552F28E0DD0FE0EA5
:10130000E66E5AEC13F0E5520028EA6AA00FE96E87
:10131000000EEA22040EEF6E4DEF13F0210EE66E82
:101320005AEC13F0E552020E0024186E0001FD5134
:10133000185C2BE2F29E8A8C939A8A9A8A9C8A8CF9
:101340008A9C8A8C8A9C8A8C8A9C002A0050EA6A31
:10135000A00FE96E000EEA22EFCF14F0002A005031
:10136000EA6AA00FE96E000EEA22EFCF13F0100E2A
:101370000D6E14321332819AD8B0818A818C819C8F
:101380000D2EF7D78A9AF28E0DD0FE0EE66E5AEC2D
:1013900013F0E5520028EA6AA00FE96E000EEA2277
:1013A000040EEF6E4DEF13F0220EE66E5AEC13F0C2
:1013B000E552F29E8A8C939A8A9A8A9C8A8A8A8CAF
:1013C0008A9C8A9A8A8C8A9C8A8C8A9C8A8C8A9C1F
:1013D0008A8C8A9C8A8C8A9C8A8C8A9C8A8C8A9C1D
:1013E0008A8C8A9C8A8C8A9C8A8C8A9C938A080E16
:1013F0000D6E818C819CD89081BAD88013320D2ECD
:10140000F8D78A9AF28E13C0E6FF5AEC13F0E55231
:101410004DEF13F0230EE66E5AEC13F0E552F29EF8
:101420008A8C939A8A9A8A9C8A8C8A9C8A8C8A9CB7
:101430008A8A8A8C8A9C8A9A8A8C8A9C8A8C8A9CC0
:101440008A8C8A9C8A8C8A9C8A8C8A9C8A8C8A9CAC
:101450008A8C8A9C8A8C8A9C938A080E0D6E818C59
:10146000819CD89081BAD88013320D2EF8D78A9AF1
:10147000F28E13C0E6FF5AEC13F0E5524DEF13F075
:10148000240EE66E5AEC13F0E552002A0050EA6A88
:10149000A00FE96E000EEA22EF500D6E0001FD5123
:1014A000005C45E201500D24186E400E185C3FE2CE
:1014B0000D50E66E5AEC13F0E552050E0DC0DBFF41
:1014C000050EDB5033E0F29E8A8C939A8A8A8A9CBE
:1014D0008A9A8A8C8A9C8A8C8A9C8A8A8A8C8A9C20
:1014E0008A9A8A8C8A9C8A8C8A9C8A8C8A9C8A8C0E
:1014F0008A9C8A8C8A9C8A8C8A9C8A8C8A9C8A8CFC
:101500008A9C938A080E0D6E818C819CD89081BA3A
:10151000D88013320D2EF8D78A9AF28E13C0E6FFC8
:101520005AEC13F0E552050EDB06CAD70DD0FE0EBD
:10153000E66E5AEC13F0E5520028EA6AA00FE96E55
:10154000000EEA22040EEF6E4DEF13F0250EE66E4C
:101550005AEC13F0E552020E0024186E0001FD5102
:10156000185C2CE2F29E8A8C939A8A9A8A9C8A8CC6
:101570008A9C8A8A8A8C8A9C8A8C8A9C002A00503F
:10158000EA6AA00FE96E000EEA22EFCF14F0002AFB
:101590000050EA6AA00FE96E000EEA22EFCF13F0C6
:1015A000100E0D6E14321332819AD8B0818A818C5C
:1015B000819C0D2EF7D78A9AF28E0DD0FE0EE66E24
:1015C0005AEC13F0E5520028EA6AA00FE96E000E0B
:1015D000EA22040EEF6E4DEF13F0260EE66E5AEC83
:1015E00013F0E552002A0050EA6AA00FE96E000EDF
:1015F000EA22EF500D6E00500D240D24186E0001EC
:10160000FD51185C36E2060E0DC0DBFF060EDB5006
:101610002FE0F29E8A8C939A8A8A8A9C8A9A8A8C74
:101620008A9C8A8A8A8C8A9C8A8C8A9C002A00508E
:10163000EA6AA00FE96E000EEA22EFCF14F0002A4A
:101640000050EA6AA00FE96E000EEA22EFCF13F015
:10165000100E0D6E14321332819AD8B0818A818CAB
:10166000819C0D2EF7D78A9AF28E060EDB06CED716
:101670000DD0FE0EE66E5AEC13F0E5520028EA6A31
:10168000A00FE96E000EEA22040EEF6E4DEF13F08C
:10169000270EE66E5AEC13F0E552040E0024186E85
:1016A0000001FD51185C65E2F29E8A8C939A8A8A49
:1016B0008A9C8A8C8A9C8A8C8A9C8A8C8A9C002A26
:1016C0000050EA6AA00FE96E000EEA22EFCF14F094
:1016D000002A0050EA6AA00FE96E000EEA22EFCF5E
:1016E00013F0100E0D6E14321332819AD8B0818A25
:1016F000818C819C0D2EF7D78A9A8A8C8A9C8A8C41
:101700008A9C8A8C8A9C8A8C002A0050EA6AA00FE4
:10171000E96E000EEA22EFCF14F0002A0050EA6AC8
:10172000A00FE96E000EEA22EFCF13F01350141051
:1017300008E000000000000000001306000E145A2C
:10174000F5D78A9CECC00DF00D5009E000000000B8
:10175000000000000000000000000D06F5D7100E8C
:101760000D6E0D5004E08A8C8A9C0D06FAD7F28E1D
:101770000DD0FE0EE66E5AEC13F0E5520028EA6A30
:10178000A00FE96E000EEA22040EEF6E4DEF13F08B
:10179000280EE66E5AEC13F0E552040E0024186E83
:1017A0000001FD51185C66E2F29E8A8C939A8A9A37
:1017B0008A9C8A8A8A8C8A9C8A8C8A9C8A8C8A9C3B
:1017C000002A0050EA6AA00FE96E000EEA22EFCF6D
:1017D00014F0002A0050EA6AA00FE96E000EEA2217
:1017E000EFCF13F0100E0D6E14321332819AD8B071
:1017F000818A818C819C0D2EF7D78A9A8A8C8A9C4B
:101800008A8C8A9C8A8C8A9C8A8C002A0050EA6A7C
:10181000A00FE96E000EEA22EFCF14F0002A00506C
:10182000EA6AA00FE96E000EEA22EFCF13F0135020
:10183000141008E000000000000000001306000E75
:10184000145AF5D78A9CECC00DF00D5009E0000049
:101850000000000000000000000000000D06F5D7A9
:10186000100E0D6E0D5004E08A8C8A9C0D06FAD77E
:10187000F28E0DD0FE0EE66E5AEC13F0E552002803
:10188000EA6AA00FE96E000EEA22040EEF6E4DEF39
:1018900013F0290EE66E5AEC13F0E552030E002405
:1018A000186E0001FD51185C36E2002A0050EA6A09
:1018B000A00FE96E000EEA22EFCF13F0F29E8A8CA1
:1018C000939A040E0D6E1332819AD8B0818A818C5E
:1018D000819C0D2EF8D7002A0050EA6AA00FE96E0D
:1018E000000EEA22EFCF14F0002A0050EA6AA00F9F
:1018F000E96E000EEA22EFCF13F0100E0D6E1432D7
:101900001332819AD8B0818A818C819C0D2EF7D7B1
:101910008A9AF28E0DD0FE0EE66E5AEC13F0E55266
:101920000028EA6AA00FE96E000EEA22040EEF6EAC
:101930004DEF13F02A0EE66E5AEC13F0E552002834
:10194000186E0001FD51185C39E2002A0050EA6A65
:10195000A00FE96E000EEA22EFCF13F0F29E8A8C00
:10196000939A040E0D6E1332819AD8B0818A818CBD
:10197000819C0D2EF8D78A8C8A9C8A8C8A9C8A8CB2
:101980008A9C8A8C8A9C8A8C8A9C8A8C8A9C8A8C67
:101990008A9C8A8C8A9C938A080E0D6E818C819C0D
:1019A000D89081BAD88013320D2EF8D78A9AF28E49
:1019B00013C0E6FF5AEC13F0E5520DD0FE0EE66EB2
:1019C0005AEC13F0E5520028EA6AA00FE96E000E07
:1019D000EA22040EEF6E4DEF13F02B0EE66E5AEC7A
:1019E00013F0E5520028186E0001FD51185C1EE24C
:1019F000002A0050EA6AA00FE96E000EEA22EF50BA
:101A00000D6EFF0E0D5C03E19368948C0ED0C70E33
:101A1000936E8A6A0DB08A860DB28A880DB48A8A5E
:101A2000949C8B9C0001050EEC6F0DD0FE0EE66EB3
:101A30005AEC13F0E5520028EA6AA00FE96E000E96
:101A4000EA22040EEF6E4DEF13F02C0EE66E5AEC08
:101A500013F0E552030E0024186E0001FD51185CCE
:101A600001E38BD0002A0050EA6AA00FE96E000E55
:101A7000EA22EF500D6E0001010E146E002A005094
:101A8000EA6AA00FE96E000EEA22EFCF13F0F3EC42
:101A900013F00D5042E0FE0E00011314E66E15EC3B
:101AA00014F0E552F7EC13F0000936E1002A00507B
:101AB000EA6AA00FE96E000EEA22EF50E66E15EC1E
:101AC00014F0E552F7EC13F0000926E137EC14F0BE
:101AD000010E00011310E66E15EC14F0E552F7EC60
:101AE00013F0000919E10001146A0D50E66E5AEC7A
:101AF00013F0E5520D500EE000EC14F0F350E66EDA
:101B00005AEC13F0E5520D50010802E252EC14F0C9
:101B10000D06F0D74CEC14F019D0010E0001131093
:101B2000E66E15EC14F0E552F7EC13F000090EE147
:101B3000010EE66E5AEC13F0E55200EC14F0F3508F
:101B4000E66E5AEC13F0E5524CEC14F0F7EC13F09F
:101B5000000910E0000114500DE0FD0EE66E5AEC95
:101B600013F0E5520028EA6AA00FE96E000EEA229F
:101B7000040EEF6E41EC14F00DD0FE0EE66E5AEC42
:101B800013F0E5520028EA6AA00FE96E000EEA227F
:101B9000040EEF6E4DEF13F02E0EE66E5AEC13F0BE
:101BA000E552040E0024186E0001FD51185C01E39B
:101BB0007FD0002A0050EA6AA00FE96E000EEA22E8
:101BC000EF500D6E0001010E146E002A0050EA6AFB
:101BD000A00FE96E000EEA22EFCF13F0F3EC13F042
:101BE000FE0E00011314E66E15EC14F0E552F7EC4E
:101BF00013F0000946E1002A0050EA6AA00FE96EDE
:101C0000000EEA22EF50E66E15EC14F0E552F7EC08
:101C100013F0000936E1002A0050EA6AA00FE96ECD
:101C2000000EEA22EF50E66E15EC14F0E552F7ECE8
:101C300013F0000926E137EC14F0010E0001131037
:101C4000E66E15EC14F0E552F7EC13F0000919E11B
:101C50000001146A0D50E66E5AEC13F0E5520D5077
:101C60000EE000EC14F0F350E66E5AEC13F0E5527F
:101C70000D50010802E252EC14F00D06F0D74CECC6
:101C800014F0F7EC13F0000910E0000114500DE01F
:101C9000FD0EE66E5AEC13F0E5520028EA6AA00F3A
:101CA000E96E000EEA22040EEF6E41EC14F00DD046
:101CB000FE0EE66E5AEC13F0E5520028EA6AA00F19
:101CC000E96E000EEA22040EEF6E4DEF13F02D0EBA
:101CD000E66E5AEC13F0E552002A0050EA6AA00FB3
:101CE000E96E000EEA22EF500D6E020E00240D2464
:101CF000186E0001FD51185C50E2F3EC13F0002A5D
:101D00000050EA6AA00FE96E000EEA22EF50FE0BC7
:101D1000E66E15EC14F0E552F7EC13F000092BE138
:101D2000002A0050EA6AA00FE96E000EEA22EF5086
:101D3000E66E15EC14F0E552F7EC13F000091BE128
:101D40000D50E66E5AEC13F0E5520D5014E0002AE7
:101D50000050EA6AA00FE96E000EEA22EF50E66E2C
:101D600015EC14F0E552F7EC13F0000902E00D68F1
:101D700002D00D06EAD70D500DE0FD0EE66E5AECCE
:101D800013F0E5520028EA6AA00FE96E000EEA227D
:101D9000040EEF6E41EC14F00DD0FE0EE66E5AEC20
:101DA00013F0E5520028EA6AA00FE96E000EEA225D
:101DB000040EEF6E4DEF13F02F0EE66E5AEC13F09B
:101DC000E5520028186E0001FD51185C3BE2002A24
:101DD0000050EA6AA00FE96E000EEA22EF500D6E85
:101DE000FF0E0D5C09E19368948C948E010E066ED3
:101DF0000001640EEC6F25D0E50E936E0DA602D0A7
:101E00008A8201D08A92949C8B9C949E0C0E0D1415
:101E10000001EC6F030E0D160D5003E1120E066E5D
:101E200010D00D0403E1080E066E0BD0020E0D5CFF
:101E300003E1050E066E05D0030E0D5C02E1020EF5
:101E4000066E0DD0FE0EE66E5AEC13F0E552002839
:101E5000EA6AA00FE96E000EEA22040EEF6E4DEF63
:101E600013F0300EE66E5AEC13F0E5520028186EAF
:101E70000001FD51185C23E2002A0050EA6AA00F1D
:101E8000E96E000EEA22EF500D6E0D50E66E5AEC30
:101E900013F0E5520D5005E1E66A5AEC13F0E552F5
:101EA0000DD093800D500AE0E66A68EC14F0E5521C
:101EB000E66E5AEC13F0E5520D06F4D70CD0FE0E88
:101EC000E66EF8DBE5520028EA6AA00FE96E000E24
:101ED000EA22040EEF6EE1D3310EE66EEBDBE55243
:101EE000002A0050EA6AA00FE96E000EEA22EF50C5
:101EF0000D6E00500D24186E0001FD51185C16E2A5
:101F00000D50E66ED7DBE552949E0D500EE0002A90
:101F10000050EA6AA00FE96E000EEA22EF50E66E6A
:101F200068EC14F0E5520D06F0D70CD0FE0EE66E0C
:101F3000C1DBE5520028EA6AA00FE96E000EEA2232
:101F4000040EEF6EAAD3320EE66EB4DBE552020E3B
:101F50000024186E0001FD51185C21E2002A005097
:101F6000EA6AA00FE96E000EEA22EF508A6E002A9C
:101F70000050EA6AA00FE96E000EEA22EF500D6EE3
:101F8000C00E0D14186E3F0E8B1418108B6E380E89
:101F90000D14186EC70E89141810896E0CD0FE0E21
:101FA000E66E88DBE5520028EA6AA00FE96E000EB3
:101FB000EA22040EEF6E71D3330EE66E7BDBE55240
:101FC000030E0024186E0001FD51185C67E2002A20
:101FD0000050EA6AA00FE96E000EEA22EF500D6E83
:101FE000002A0050EA6AA00FE96E000EEA22EFCF45
:101FF00014F0002A0050EA6AA00FE96E000EEA22EF
:10200000EFCF13F001500D240D24186E400E185C14
:1020100038E20D50E66E4EDBE5520D5031E0200EF9
:10202000E66E68EC14F0E55214C0E6FF68EC14F0BC
:10203000E55213C0E6FF68EC14F0E552E66A68EC7E
:1020400014F0E552E66E36DBE552280EE66E68ECDB
:1020500014F0E55214C0E6FF68EC14F0E55213C02A
:10206000E6FF68EC14F0E552E66A68EC14F0E5521D
:10207000E66E20DBE552132A000E14220D06CDD7A2
:102080000CD0FE0EE66E16DBE5520028EA6AA00FC1
:10209000E96E000EEA22040EEF6E0CD0FE0EE66E24
:1020A00009DBE5520028EA6AA00FE96E000EEA2279
:1020B000040EEF6EF2D2340EE66EFCDAE552002A20
:1020C0000050EA6AA00FE96E000EEA22EF500D6E92
:1020D00000500D240D24020F186E0001FD51185CF4
:1020E0004CE20D50E66EE6DAE552002A0050EA6A4C
:1020F000A00FE96E000EEA22EFCF14F0002A005084
:10210000EA6AA00FE96E000EEA22EFCF13F00D503D
:1021100033E0400EE66EDCDBE55214C0E6FFD8DBB0
:10212000E55213C0E6FFD4DBE552002A0050EA6A0C
:10213000A00FE96E000EEA22EF50E66EC9DBE55211
:10214000480EE66EC5DBE55214C0E6FFC1DBE55282
:1021500013C0E6FFBDDBE552002A0050EA6AA00F7B
:10216000E96E000EEA22EF50E66EB2DBE552132A6A
:10217000000E14220D06CBD70CD0FE0EE66E9ADAB6
:10218000E5520028EA6AA00FE96E000EEA22040E6A
:10219000EF6E83D2350EE66E8DDAE5520028186EAA
:1021A0000001FD51185C11E2002A0050EA6AA00FFC
:1021B000E96E000EEA22EF500D6EFF0E0D5C02E19B
:1021C0008A9602D093968A860CD0FE0EE66E72DA5C
:1021D000E5520028EA6AA00FE96E000EEA22040E1A
:1021E000EF6E5BD2360EE66E65DAE552030E002422
:1021F000186E0001FD51185C35E2F29E939A8A9A9E
:102200008A8C8A9C8A8C8A9C8A8C8A9C8A8C8A9CDE
:10221000002A0050EA6AA00FE96E000EEA22EFCF12
:1022200014F0002A0050EA6AA00FE96E000EEA22BC
:10223000EFCF13F0002A0050EA6AA00FE96E000EFB
:10224000EA22EF500E6E180E0D6E143213320E325B
:10225000819AD8B0818A818C819C0D2EF6D78A9A7A
:10226000F28E0CD0FE0EE66E25DAE5520028EA6A00
:10227000A00FE96E000EEA22040EEF6E0ED2370EAA
:10228000E66E18DAE552F29E939A8A8A8A8C8A9CC4
:102290008A9A0D6A0B0E0D5C04E28A8C8A9C0D2AC8
:1022A000F9D7938A100E0D6E818CD89081BAD880A0
:1022B00014321332819C0D2EF7D78A9AF28E14C0F5
:1022C000E6FFF8D9E55213C0E6FFF4D9E552E5D1AF
:1022D000380EE66EEFD9E552F29E939A8A9A0D6A0D
:1022E0001C0E0D5C04E28A8C8A9C0D2AF9D7F28EB2
:1022F000D4D1390EE66EDED9E552002A0050EA6AE2
:10230000A00FE96E000EEA22EF500D6E00500D2472
:102310000D24186E0001FD51185C2CE2F29E939A78
:10232000070E0DC0DBFF070EDB5020E0002A005037
:10233000EA6AA00FE96E000EEA22EFCF14F0002A3D
:102340000050EA6AA00FE96E000EEA22EFCF13F008
:10235000100E0D6E13361436819AD8B0818A818C96
:10236000819C0D2EF7D7070EDB06DDD78A9A938A5C
:10237000F28E0CD0FE0EE66E9DD9E5520028EA6A78
:10238000A00FE96E000EEA22040EEF6E86D13A0E1F
:10239000E66E90D9E552002A0050EA6AA00FE96E75
:1023A000000EEA22EF500D6E0001FD51005C2BE2A1
:1023B00001500D240D24186E400E185C24E20D50BF
:1023C000E66E78D9E552F29E938A080E0DC0DBFFC7
:1023D000080EDB5016E0100E0D6E818CD89081BA7D
:1023E000D88013361436819C0D2EF7D714C0E6FF23
:1023F00061D9E55213C0E6FF5DD9E552080EDB0650
:10240000E7D7F28E0CD0FE0EE66E54D9E5520028C6
:10241000EA6AA00FE96E000EEA22040EEF6E3DD1CB
:102420003B0EE66E47D9E552C50E936E8A6A949EBE
:1024300034D13C0EE66E3ED9E552002A0050EA6ADD
:10244000A00FE96E000EEA22EF500D6E0D0400247D
:10245000E8380F0B186E0001FD51185C21E2F29E66
:102460000E6A0D5000081AE20E500BE1002A0050CF
:10247000EA6AA00FE96E000EEA22EFCF13F0080E11
:102480000E6E1336829ED8B0828E818200000000CC
:102490000000000081920D060E06E3D7F28E0CD0EC
:1024A000FE0EE66E07D9E5520028EA6AA00FE96E33
:1024B000000EEA22040EEF6EF0D03D0EE66EFAD862
:1024C000E5520028186E0001FD51185C34E20D043D
:1024D0000124E8380F0B196E400E195C2CE2002A1B
:1024E0000050EA6AA00FE96E000EEA22EF500D6E6E
:1024F0000D50E66EDFD8E552F29E080E0E6E0D50BE
:10250000000817E2818200000000000000008192B4
:10251000D89081B0D88013360E060E5002E00D041C
:1025200006E1080E0E6E13C0E6FFC4D8E5520D0694
:10253000E6D7F28E0CD0FE0EE66EBCD8E55200282F
:10254000EA6AA00FE96E000EEA22040EEF6EA5D033
:10255000400E015C09E20150EA6A600FE96E000E6C
:10256000EA22EF6A012AF4D7016A04010CBF0BD0FA
:10257000400EE66E600EE66E000EE66EA0EC14F005
:10258000E552E552E552006888D0F00EE66E92D82A
:10259000E552020E0024186E0001FD51185C25E280
:1025A000002A0050EA6AA00FE96E000EEA22EFCF7F
:1025B00014F0002A0050EA6AA00FE96E000EEA2229
:1025C000EFCF13F014C0E6FF75D8E55213C0E6FF55
:1025D00071D8E55214C0EAFF13C0E9FFEF500D6E49
:1025E0000D50E66E67D8E5520CD0FE0EE66E62D84E
:1025F000E5520028EA6AA00FE96E000EEA22040EF6
:10260000EF6E4BD0F10EE66E55D8E552030E002466
:10261000186E0001FD51185C2EE2002A0050EA6A93
:10262000A00FE96E000EEA22EFCF14F0002A00504E
:10263000EA6AA00FE96E000EEA22EFCF13F0002A3B
:102640000050EA6AA00FE96E000EEA22EF500D6E0C
:1026500014C0E6FF2FD8E55213C0E6FF2BD8E55291
:102660000D50E66E27D8E55214C0EAFF13C0E9FF0B
:102670000D50EF6E0CD0FE0EE66E1CD8E552002811
:10268000EA6AA00FE96E000EEA22040EEF6E05D092
:10269000FE0EE66E0FD8E55200D0002A01D08992D6
:1026A000090EE15C02E2E16AE552E16EE552E7CF34
:1026B000D9FF1200D9CFE6FFE1CFD9FF0001EA51DF
:1026C0000AE00A0E025C11E20250022AEA6AE00FF6
:1026D000E96E000E06D00150012AEA6A600FE96E29
:1026E000000EEA22FE0EDBCFEFFF400E015C13E18D
:1026F000016A04010CBF0CD0400EE66E600EE66E5F
:10270000000EE66EA0EC14F0E552E552E55203D05F
:102710000001010EEA6FE552E7CFD9FF1200D8CFD2
:10272000E4FFE0CFE4FFE46EDACFE4FFE2CFDAFFCC
:10273000F3CFE4FFF4CFE4FFE652C282F40ECF6E93
:10274000480ECE6EC2B2FED79E9007C009F008C0F8
:102750000AF0C4CF08F0C3CF07F00B50075E0C504F
:10276000085AE10E0902F4CF10F0F3CF0FF0E10E9A
:102770000A02F35010260F50032610500422E40ED4
:102780000702F4CF10F0F3CF0FF0E40E0802F3507D
:1027900010260F50035E1050045A0001043402E367
:1027A000036A046A05500001D880045402E205C09F
:1027B00004F004C0BEFF00010350E840E8403F0BB6
:1027C000300B1E6ECF0EBD141E10BD6EE552E5CF50
:1027D000F4FFE5CFF3FFE5CFDAFFE550E5CFE0FF0B
:1027E000E5CFD8FF10008A90939059EF14F08A92A9
:1027F000939293805ED893825CD881B0FF0C000CDA
:10280000080E166E8A929392938053D8938251D871
:10281000159E1546159081B015801606F4E1196ACB
:1028200015C0F3FF19C0F4FF1200D9CFE6FFE1CFC6
:10283000D9FF080E166EFE0EDB50156E8A92153704
:10284000D8A006D09392938034D8938232D806D001
:1028500093928A9093902DD893822BD81606165077
:10286000EEE1000E00D0E552E7CFD9FF12008A92C8
:10287000939293801ED893821CD88A90939059EF9C
:1028800014F08A9293928A90939013D8938211D8DD
:1028900093800FD859EF14F0939293800AD89382C3
:1028A00059EF14F093928A90939003D8938259EF42
:1028B00014F0ECC017F0175009E000000000000011
:1028C00000000000000000001706F5D700D012003D
:1028D000D9CFE6FFE1CFD9FFF29EFE0EDB50156E99
:1028E000ECC00FF0080E0E6E0FB404D015AE829E31
:1028F00015BE828E0650176E172EFED70FA6818248
:102900000FB681920FA405D015AE829E15BE828EA1
:1029100002D0813015360650176E172EFED70FA63F
:1029200081920FB681820FA402D0813015360E2E0F
:10293000DBD7F28E155000D0E552E7CFD9FF120059
:10294000D9CFE6FFE1CFD9FFE65204010CAF02D0A8
:10295000000E33D0FC0EDB50400805E2400EF36E53
:10296000FC0EF3CFDBFFDF6AFC0EDB50DF5C19E20D
:10297000DF50E76EFD0EDBCFE9FFFE0EDBCFEAFF97
:10298000E750E926000EEA22EF50E66EDF50EA6AD1
:10299000680FE96E040EEA22E552E750EF6EDF2A77
:1029A000E3D7FC0EDBCF0DF404010CAD02D0880E92
:1029B00001D0C80E0C6FFC0EDB50E552E552E7CF9C
:1029C000D9FF1200D9CFE6FFE1CFD9FF0101536B48
:1029D000040108BF32D0FC0EDBCF18F00951D880BB
:1029E000185403E2FC0E09C4DBFF0101536BFC0E1B
:1029F000DB50535D19E25351EA6A280FE96E040E69
:102A0000EA22EF50E66E5351E76EFD0EDBCFE9FF91
:102A1000FE0EDBCFEAFFE750E926000EEA22E55280
:102A2000E750EF6E532BE3D70401400E096F08AD5A
:102A300002D0880E01D0C80E086F01015351E55233
:102A4000E7CFD9FF12000101536B1E0E716E040116
:102A5000400E096F280E186E040E18C00AF40B6F92
:102A6000880E086F680E186E040E18C00EF40F6FF3
:102A7000400E0C6F1200D9CFE6FFE1CFD9FFE6522E
:102A800012C4DFFF0101010E476FE552E552E7CFA7
:102A9000D9FF1200D9CFE6FFE1CFD9FFE65212C429
:102AA000DFFF0101010E476FE552E552E7CFD9FF85
:102AB0001200D9CFE6FFE1CFD9FF020EE1261F0EAB
:102AC00004011015010865E1145163E111C4DFFF31
:102AD000060EDF5C23E1010E13C4DBFFDB5021088F
:102AE00009E10101010E476F090E4A6F330E4B6F6A
:102AF000090E0CD0010EDB5022080DE10101010E80
:102B0000476F290E4A6F330E4B6F220E4E6F4F6B7D
:102B1000010E506F03D0010EDB502308600E04013C
:102B20001015200836E1DF0402E1A5DF32D0090EDE
:102B3000DF5C05E10101010E466FACDF2AD0020E19
:102B4000DF5C07E10101010E476F510E486F010E76
:102B500012D00A0EDF5C06E10101010E476F13C4BB
:102B600051F117D0030EDF5C0CE10101010E476F3C
:102B7000520E486F010E496F010E4E6F4F6B506B36
:102B800008D00B0EDF5C05E10101010E476F12C496
:102B900052F1020EE15C02E2E16AE552E16EE552B9
:102BA000E7CFD9FF1200D9CFE6FFE1CFD9FF020E60
:102BB000E126800E0401105D3CE113C4DFFF010E2D
:102BC00012C4DBFFDF0409E10101010E476FEE0EC5
:102BD0004A6F320E4B6F120E28D0020EDF5C09E1F5
:102BE0000101010E476F000E4A6F330E4B6F290E25
:102BF0001CD0030EDF5C1DE10101010E476FDB50AD
:102C000004E14B0E4A6F330E0AD0010EDB0404E1DF
:102C10004F0E4A6F330E03D06F0E4A6F330E4B6F59
:102C20004AC1F6FFF76E0800F5504E6F4F6B010E6C
:102C3000506F020EE15C02E2E16AE552E16EE5529C
:102C4000E7CFD9FF1200D9CFE6FFE1CFD9FF030EBE
:102C5000E1261F0E04011015DF6E206B216BDF5083
:102C60000DE10101010E476F435102E00401208193
:102C70000101415135E00401208332D0DF0404E139
:102C80000101010E476F2CD0020EDF5C29E10F0E0F
:102C90001415E76E010EE7CFDBFF800E1415E76E0B
:102CA000020EE7CFDBFF0101010E476FDB50080D7D
:102CB000F3504C6F4D6B000E4C27040E4D23020E4B
:102CC000DB5004E0040E4C27000E4D234CC1E9FFFD
:102CD0004DC1EAFFEF50040B03E00401010E206F29
:102CE0000101475108E0200E486F040E496F020EA3
:102CF0004E6F4F6B506B030EE15C02E2E16AE552EE
:102D0000E16EE552E7CFD9FF1200D9CFE6FFE1CF60
:102D1000D9FF040EE1261F0E04011015DF6E010E0F
:102D200012C4DBFFDF5011E1010EDB044CE10101B5
:102D3000010E476F030E0401115D04E10101010E54
:102D4000416F41D00101416B3ED0020EDF5C3BE19F
:102D50000F0E1415E76E020EE7CFDBFF800E141581
:102D6000E76E030EE7CFDBFF010EDB502CE1020E16
:102D7000DB5029E00101010E476F020EDB50080D08
:102D8000F3504C6F4D6B000E4C27040E4D23030E79
:102D9000DB5004E0040E4C27000E4D23030E04010B
:102DA000115D02E1840E0AD0030EDB0406E14CC182
:102DB000E9FF4DC1EAFFEF6A06D0880E4CC1E9FF7A
:102DC0004DC1EAFFEF6E040EE15C02E2E16AE552FA
:102DD000E16EE552E7CFD9FF1200D9CFE6FFE1CF90
:102DE000D9FFE65211C4DFFF600E0401101554E153
:102DF000050EDF5C08E10101010E476F040E406F14
:102E000012C442F149D0060EDF5C02E1CCDE44D0B0
:102E1000090EDF5C0EE10101010E476F12C444F19F
:102E2000445103E1040E406F37D0050E406F0BDEB6
:102E300033D0080EDF5C07E10101010E476F440E3D
:102E4000486F010E17D0DF5002E1FDDE25D0DF0410
:102E500003E0030EDF5C02E158DF1ED00A0EDF5CE8
:102E60000FE10101010E476F0401206B0101200EEB
:102E7000486F040E496F010E4E6F4F6B506B0CD0B4
:102E80000B0EDF5C04E10101010E476F05D0070E58
:102E9000DF5C02E00C0EDF5CE552E552E7CFD9FFC4
:102EA0001200D9CFE6FFE1CFD9FF030EE1260101E1
:102EB000080E4E5D000E4F5907E2010E4EC1DBFFBA
:102EC000020E4FC1DBFF07D0080EF36E010EF3CFE9
:102ED000DBFF020EDB6AFC0E04010417010E020E7A
:102EE000DBCF19F0000E030E191619C018F0195097
:102EF0000413FF0EE76E010EDBCF18F0020EE75051
:102F0000181618C005F4200E186E040E1B6A18C09F
:102F100006F4076F010EDB5001014E5F020EDB501D
:102F20004F5B200E4C6F040E4D6F500524E1DF6A9D
:102F3000DFCF18F0010EDBCF19F0020EDBCF1AF055
:102F40001950185C000E1A5439E24AC1F6FF4BC101
:102F5000F7FF4A2B000E4B230800F550E66E4CC1DC
:102F6000E9FF4DC1EAFF4C2B000E4D23E552E7501F
:102F7000EF6EDF2ADDD7DF6ADFCF18F0010EDBCF7F
:102F800019F0020EDBCF1AF01950185C000E1A541B
:102F900015E248C1E9FF49C1EAFF482B000E492369
:102FA000EF50E66E4CC1E9FF4DC1EAFF4C2B000E1D
:102FB0004D23E552E750EF6EDF2ADED7030EE15CCA
:102FC00002E2E16AE552E16EE552E7CFD9FF120075
:102FD000D9CFE6FFE1CFD9FF040EE1260401F3507B
:102FE0000111E66ED950020FE96EDACFEAFFE55221
:102FF000E750EE6EED6A020EDB5001014E27030E24
:10300000DB504F23200E486F040E496FDE6ADD6AE5
:10301000DECF18F0DDCF19F0020EDBCF1AF0030E71
:10302000DBCF1BF01A50185C1B50195818E248C12E
:10303000E9FF49C1EAFF482B000E4923EF50E66E35
:103040004CC1E9FF4DC1EAFF4C2B000E4D23E55268
:10305000E750EF6EDF2A010EDBE3DB2AD9D7040E3F
:10306000E15C02E2E16AE552E16EE552E7CFD9FFA9
:1030700012000401049F009F0101456B476B466BE2
:103080004E6B4F6BAADE15DD010147510EE10401C5
:10309000080E016F100E186E040E1A6A1B6A18C013
:1030A00002F4036F840E006F30D0040110AF2FD0F4
:1030B00001014E510401165D01014F5104011759E0
:1030C00004E216C44EF117C44FF1EBDE0101020E0B
:1030D000456F0401080E016F100E186E040E196E74
:1030E0001A6A1B6A1A6A1B6A18C002F4036F800E00
:1030F000006F200E186E040E196E1A6A1B6A1A6A87
:103100001B6A18C006F4076FC80E046F16D00101C1
:10311000010E456F0401056BC80E046F080E016FA8
:10312000200E186E040E196E1A6A1B6A1A6A1B6A40
:1031300018C002F4036FC80E006F6D9812000101F1
:10314000456B0401080E016F100E186E040E18C0B6
:1031500002F4036F880E006F046B1200D9CFE6FFF4
:10316000E1CFD9FF020EE1266C5024E13C0E0401B0
:103170000015E840E8403F0BDF6E0D0EDF5C02E11A
:1031800078DF35D00101450531E122DF01014651EB
:1031900009E0010E12C4DBFF020E0401135D02E020
:1031A000030E135D040100AD02D0880E01D0C80EDD
:1031B000006F1DD0040E6C5C1AE16E500AE1040E23
:1031C0000101405D06E112C46EFF6E5002E1030E84
:1031D000406F020E0101455D09E163DE040104ADAB
:1031E00002D0880E01D0C80E046F01D0A8DF020EF5
:1031F000E15C02E2E16AE552E16EE552E7CFD9FF18
:1032000012006DB606D06D6A696A6D860101010E05
:10321000406F0101400509E16D50200B06E1686A2D
:10322000696A69806988020E406F12006D92699424
:1032300068941200689C120070A002D080DF709029
:10324000689A120012006A6A686A9F0E6B6E7B0EA3
:10325000696E6E6A160E706E68A602D06896FCD70C
:103260006D986DDF0101416B436B446B030E406F42
:1032700012000101405101E112006850040B04E00A
:103280006950040B01E0D2DF6DB212006850010BEF
:1032900004E06950010B01E0D6DF6850100B04E038
:1032A0006950100B01E0CEDF6850400B04E069501C
:1032B000400B01E0BFDF6850200B04E06950200B99
:1032C00001E0BADF6850020B04E06950020B01E034
:1032D0006892030E0101405D01E212006850080B84
:0E32E00005E06950080B02E039DF6896120025
:0232EE001201CB
:1032F000000200000008D8040001010001020001E2
:1033000009022900010100A03209040000020300A3
:10331000000009210101000122220007058103406C
:1033200000010705010340000106A0FF0901A101FA
:103330000903150026FF0075089540810209041550
:103340000026FF00750895409102C004030904207F
:10335000034F00700065006E002000500072006F87
:10336000006700720061006D006D00650072003E34
:10337000034F00700065006E002000500072006F67
:10338000006700720061006D006D00650072002032
:10339000002000550053004200200048004900442E
:0D33A00000200063006C00610073007300EA
:0133AD00001F
:0233AE002A0EE5
:1033B000F66E000EF76E000EF86E00010900F55073
:1033C000F86F0900F550F96F03E1F86701D03DD0BF
:1033D0000900F550F36F0900F550F46F0900F5503E
:1033E000F56F09000900F550E96E0900F550EA6E25
:1033F000090009000900F550F66F0900F550F76F54
:1034000009000900F6CFFAF0F7CFFBF0F8CFFCF097
:10341000F3C0F6FFF4C0F7FFF5C0F8FF0001F65364
:1034200002E1F75307E00900F550EE6EF607F8E207
:10343000F707F9D7FAC0F6FFFBC0F7FFFCC0F8FFAB
:0C3440000001F807000EF95BBFD7120076
:04344C000F0EC1128C
:10345000140E6F6E0101406B0101416B0101446B61
:1034600022EC00F001EC19F06FBE02D039EC19F03B
:0634700061EC00F0F7D74B
:0A34760011EE00F021EE00F0F86AFC
:103480001D9CD7EC19F050EC1AF026EC1AF0FBD783
:02349000120028
:0E34920000EE00F00F0EEE6AEA62FDD71200A7
:0234A000120018
:0E34A2000000000000640100000000AB030009
:0A34B0000000000000000000000012
:020000040030CA
:0100000022DD
:010001000EF0
:010002003DC0
:010003001EDE
:0100050000FA
:010006008178
:00000001FF
